:020000040000FA
:020000000528D1
:08000800090007309F0086018A
:1000100085018316DF30810002308600E0308500E4
:100020001930990018159816831218169817312050
:10003000803090202310981C1F28181218168C1E30
:100040001B281A08A000A00F272823141B28A00F84
:100050002B2823101B2823182F2890201B289E2094
:100060001B2886019630AE20303086006B20293068
:10007000AE206B200130AE20203086006B20013096
:10008000AE20203086006B200130AE20803086000C
:100090006B200130AE20003086006B200130AE2096
:1000A000803086006B200130AE20003086006B204F
:1000B0000130AE20E03086006B200130AE200030F1
:1000C00086006B200130AE20603086006B2001304E
:1000D000AE2071200034861500000000000086115B
:1000E0000034003086006B200130AE2010308600D6
:1000F0006B203230AE20003086006B200130AE2005
:10010000603086006B200130AE20003086006B200E
:100110000130AE20C03086006B200130AE200034AC
:10012000A000F030200586006B200130AE20200EAC
:10013000F03986006B200130AE200800A000F030BE
:100140002005013886006B200130AE20200EF039EA
:10015000013886006B200130AE200800A2001E305E
:10016000A100A10BB1280000A20BB82800000034A8
:060170000000BA28AF28D0
:02400E00423F2F
:00000001FF
